BL51 BANKED LINKER/LOCATER V6.22                                                        11/30/2016  13:53:19  PAGE 1


BL51 BANKED LINKER/LOCATER V6.22, INVOKED BY:
E:\KEIL_V5\C51\BIN\BL51.EXE .\Objects\STARTUP.obj, .\Objects\main.obj, .\Objects\game.obj, .\Objects\malloc.obj, .\Objec
>> ts\tftlcd.obj, .\Objects\74HC165.obj TO .\Objects\RAM PRINT (.\Listings\RAM.m51) RAMSIZE (256) DISABLEWARNING (16)


MEMORY MODEL: LARGE


INPUT MODULES INCLUDED:
  .\Objects\STARTUP.obj (?C_STARTUP)
  .\Objects\main.obj (MAIN)
  .\Objects\game.obj (GAME)
  .\Objects\malloc.obj (MALLOC)
  .\Objects\tftlcd.obj (TFTLCD)
  .\Objects\74HC165.obj (74HC165)
  E:\KEIL_V5\C51\LIB\C51L.LIB (?C_INIT)
  E:\KEIL_V5\C51\LIB\C51L.LIB (?C?SCDIV)
  E:\KEIL_V5\C51\LIB\C51L.LIB (?C?CLDPTR)
  E:\KEIL_V5\C51\LIB\C51L.LIB (?C?CSTPTR)
  E:\KEIL_V5\C51\LIB\C51L.LIB (?C?IMUL)
  E:\KEIL_V5\C51\LIB\C51L.LIB (?C?SIDIV)
  E:\KEIL_V5\C51\LIB\C51L.LIB (?C?IILDX)
  E:\KEIL_V5\C51\LIB\C51L.LIB (?C?ILDIX)
  E:\KEIL_V5\C51\LIB\C51L.LIB (?C?ILDOPTR)
  E:\KEIL_V5\C51\LIB\C51L.LIB (?C?ISTOPTR)
  E:\KEIL_V5\C51\LIB\C51L.LIB (?C?LMUL)
  E:\KEIL_V5\C51\LIB\C51L.LIB (?C?ULDIV)
  E:\KEIL_V5\C51\LIB\C51L.LIB (?C?ULCMP)
  E:\KEIL_V5\C51\LIB\C51L.LIB (?C?LLDIXDATA)
  E:\KEIL_V5\C51\LIB\C51L.LIB (?C?LSTXDATA)
  E:\KEIL_V5\C51\LIB\C51L.LIB (?C?LSTKXDATA)
  E:\KEIL_V5\C51\LIB\C51L.LIB (?C?ICALL)
  E:\KEIL_V5\C51\LIB\C51L.LIB (VSPRINTF)
  E:\KEIL_V5\C51\LIB\C51L.LIB (?C?UIDIV)
  E:\KEIL_V5\C51\LIB\C51L.LIB (PRINTF)
  E:\KEIL_V5\C51\LIB\C51L.LIB (?C?CLDOPTR)
  E:\KEIL_V5\C51\LIB\C51L.LIB (?C?PLDIXDATA)
  E:\KEIL_V5\C51\LIB\C51L.LIB (?C?PSTXDATA)
  E:\KEIL_V5\C51\LIB\C51L.LIB (?C?CCASE)
  E:\KEIL_V5\C51\LIB\C51L.LIB (PUTCHAR)


LINK MAP OF MODULE:  .\Objects\RAM (?C_STARTUP)


            TYPE    BASE      LENGTH    RELOCATION   SEGMENT NAME
            -----------------------------------------------------

            * * * * * * *   D A T A   M E M O R Y   * * * * * * *
            REG     0000H     0008H     ABSOLUTE     "REG BANK 0"
            DATA    0008H     0005H     UNIT         ?DT?PRINTF?PRINTF
                    000DH     0013H                  *** GAP ***
            BIT     0020H.0   0001H.1   UNIT         ?BI?PRINTF?PRINTF
                    0021H.1   0000H.7                *** GAP ***
            IDATA   0022H     0001H     UNIT         ?STACK

            * * * * * * *  X D A T A   M E M O R Y  * * * * * * *
            XDATA   0000H     1C00H     ABSOLUTE     
BL51 BANKED LINKER/LOCATER V6.22                                                      11/30/2016  13:53:19  PAGE 2


            XDATA   1C00H     01C0H     ABSOLUTE     
            XDATA   1DC0H     003EH     UNIT         _XDATA_GROUP_
            XDATA   1DFEH     0031H     UNIT         ?XD?_LCD_PRINTF?TFTLCD
            XDATA   1E2FH     0028H     UNIT         ?XD?PRINTF?PRINTF
            XDATA   1E57H     0019H     UNIT         ?XD?MALLOC
            XDATA   1E70H     0014H     UNIT         ?XD?TFTLCD
            XDATA   1E84H     0010H     UNIT         ?XD?_MYMEMCPY?MALLOC
            XDATA   1E94H     000CH     UNIT         ?XD?_MYREALLOC?MALLOC
            XDATA   1EA0H     000BH     UNIT         ?XD?GAME
            XDATA   1EABH     000BH     UNIT         ?XD?_MEM_FREE?MALLOC
            XDATA   1EB6H     000AH     UNIT         ?XD?_LCDDRAWCIRCLE?TFTLCD
            XDATA   1EC0H     0008H     UNIT         ?XD?_MYFREE?MALLOC
            XDATA   1EC8H     0006H     UNIT         ?XD?_VSPRINTF?VSPRINTF

            * * * * * * *   C O D E   M E M O R Y   * * * * * * *
            CODE    0000H     0003H     ABSOLUTE     
            CODE    0003H     17C0H     UNIT         ?CO?TFTLCD
            CODE    17C3H     0830H     UNIT         ?PR?_LCDDRAWCIRCLEA?TFTLCD
            CODE    1FF3H     0394H     UNIT         ?C?LIB_CODE
            CODE    2387H     0365H     UNIT         ?PR?PRINTF?PRINTF
            CODE    26ECH     0265H     UNIT         ?PR?_MEM_MALLOC?MALLOC
            CODE    2951H     025BH     UNIT         ?PR?GAMESTART?GAME
            CODE    2BACH     0241H     UNIT         ?PR?_LCDDRAWCIRCLE?TFTLCD
            CODE    2DEDH     020CH     UNIT         ?PR?_LCDDRAWLINE?TFTLCD
            CODE    2FF9H     01D3H     UNIT         ?PR?_ISFIVECHESSCONTANT?GAME
            CODE    31CCH     01BAH     UNIT         ?PR?_GETCHESSNUM?GAME
            CODE    3386H     01B4H     UNIT         ?PR?_LCDDISPSTRING?TFTLCD
            CODE    353AH     015FH     UNIT         ?PR?_LCDDISPCHAR?TFTLCD
            CODE    3699H     0132H     UNIT         ?PR?_MEM_FREE?MALLOC
            CODE    37CBH     0112H     UNIT         ?PR?DRAWCHESSBOARD?GAME
            CODE    38DDH     0104H     UNIT         ?PR?_MYREALLOC?MALLOC
            CODE    39E1H     00F7H     UNIT         ?PR?RETRACTCHESS?GAME
            CODE    3AD8H     00F5H     UNIT         ?PR?_MEM_PERUSED?MALLOC
            CODE    3BCDH     00F1H     UNIT         ?PR?_DRAWCHESS?GAME
            CODE    3CBEH     00E1H     UNIT         ?PR?_LCDDRAWRECT?TFTLCD
            CODE    3D9FH     00CDH     UNIT         ?PR?_LCD_PRINTF?TFTLCD
            CODE    3E6CH     00A4H     UNIT         ?PR?_MEM_INIT?MALLOC
            CODE    3F10H     0098H     UNIT         ?PR?_LCDFILL?TFTLCD
            CODE    3FA8H     0093H     UNIT         ?PR?_CLEARCHESS?GAME
            CODE    403BH     008CH     UNIT         ?C_C51STARTUP
            CODE    40C7H     0080H     UNIT         ?PR?RESSTART?GAME
            CODE    4147H     0079H     UNIT         ?PR?_MYFREE?MALLOC
            CODE    41C0H     0079H     UNIT         ?PR?_MYMALLOC?MALLOC
            CODE    4239H     0068H     UNIT         ?PR?_CLEARSELECTBOX?GAME
            CODE    42A1H     005FH     UNIT         ?PR?_DRAWSELECTBOX?GAME
            CODE    4300H     0059H     UNIT         ?PR?_MYMEMCPY?MALLOC
            CODE    4359H     0052H     UNIT         ?PR?_LCDCLEAR?TFTLCD
            CODE    43ABH     004AH     UNIT         ?C_INITSEG
            CODE    43F5H     004AH     UNIT         ?PR?_VSPRINTF?VSPRINTF
            CODE    443FH     003FH     UNIT         ?PR?_LCDDRAWPOINT?TFTLCD
            CODE    447EH     003AH     UNIT         ?PR?_MYMEMSET?MALLOC
            CODE    44B8H     0035H     UNIT         ?CO?GAME
            CODE    44EDH     0031H     UNIT         ?PR?GAMEINIT?GAME
            CODE    451EH     002AH     UNIT         ?PR?_LCDSETPOS?TFTLCD
            CODE    4548H     0027H     UNIT         ?PR?PUTCHAR?PUTCHAR
            CODE    456FH     0024H     UNIT         ?PR?HC165_READ?74HC165
            CODE    4593H     0020H     UNIT         ?PR?LCDREADDATA?TFTLCD
BL51 BANKED LINKER/LOCATER V6.22                                                      11/30/2016  13:53:19  PAGE 3


            CODE    45B3H     001FH     UNIT         ?PR?_ISGAMEOVER?GAME
            CODE    45D2H     001DH     UNIT         ?PR?_DELAY_MS?TFTLCD
            CODE    45EFH     0019H     UNIT         ?PR?MAIN?MAIN
            CODE    4608H     0016H     UNIT         ?PR?_LCDWRITECOM?TFTLCD
            CODE    461EH     0010H     UNIT         ?PR?_LCDWRITEDATA?TFTLCD
            CODE    462EH     000EH     UNIT         ?PR?_DELAY_US?TFTLCD
            CODE    463CH     0009H     UNIT         ?PR?_LCDSETBKCOLOR?TFTLCD
            CODE    4645H     0009H     UNIT         ?PR?_LCDSETCOLOR?TFTLCD



OVERLAY MAP OF MODULE:   .\Objects\RAM (?C_STARTUP)


SEGMENT                                XDATA_GROUP
  +--> CALLED SEGMENT                START    LENGTH
----------------------------------------------------
?C_C51STARTUP                        -----    -----
  +--> ?PR?MAIN?MAIN
  +--> ?C_INITSEG

?PR?MAIN?MAIN                        -----    -----
  +--> ?PR?GAMEINIT?GAME
  +--> ?PR?GAMESTART?GAME

?PR?GAMEINIT?GAME                    -----    -----
  +--> ?PR?_MYMALLOC?MALLOC
  +--> ?PR?_LCDCLEAR?TFTLCD
  +--> ?PR?DRAWCHESSBOARD?GAME
  +--> ?PR?_DRAWSELECTBOX?GAME

?PR?_MYMALLOC?MALLOC                 1DC0H    0009H
  +--> ?PR?_MEM_MALLOC?MALLOC

?PR?_MEM_MALLOC?MALLOC               1DC9H    0011H

?PR?_LCDCLEAR?TFTLCD                 1DC0H    0002H
  +--> ?PR?_LCDWRITECOM?TFTLCD
  +--> ?PR?_LCDWRITEDATA?TFTLCD

?PR?DRAWCHESSBOARD?GAME              1DC5H    0002H
  +--> ?PR?_LCDFILL?TFTLCD
  +--> ?PR?_LCDSETCOLOR?TFTLCD
  +--> ?PR?_LCDDRAWRECT?TFTLCD
  +--> ?PR?_LCDDRAWLINE?TFTLCD

?PR?_LCDFILL?TFTLCD                  1DC7H    000EH
  +--> ?PR?_LCDSETPOS?TFTLCD
  +--> ?PR?_LCDWRITEDATA?TFTLCD

?PR?_LCDSETPOS?TFTLCD                -----    -----
  +--> ?PR?_LCDWRITECOM?TFTLCD

?PR?_LCDDRAWRECT?TFTLCD              1DC9H    0008H
  +--> ?PR?_LCDDRAWLINE?TFTLCD

?PR?_LCDDRAWLINE?TFTLCD              1DDEH    001EH
BL51 BANKED LINKER/LOCATER V6.22                                                      11/30/2016  13:53:19  PAGE 4


  +--> ?PR?_LCDDRAWPOINT?TFTLCD

?PR?_LCDDRAWPOINT?TFTLCD             1DFCH    0002H
  +--> ?PR?_LCDWRITECOM?TFTLCD
  +--> ?PR?_LCDWRITEDATA?TFTLCD

?PR?_DRAWSELECTBOX?GAME              1DC5H    0004H
  +--> ?PR?_LCDSETCOLOR?TFTLCD
  +--> ?PR?_LCDDRAWRECT?TFTLCD

?PR?GAMESTART?GAME                   1DC0H    0001H
  +--> ?PR?HC165_READ?74HC165
  +--> ?PR?_CLEARSELECTBOX?GAME
  +--> ?PR?_DRAWSELECTBOX?GAME
  +--> ?PR?_DRAWCHESS?GAME
  +--> ?PR?_ISGAMEOVER?GAME
  +--> ?PR?_LCDSETCOLOR?TFTLCD
  +--> ?PR?_LCDFILL?TFTLCD
  +--> ?CO?GAME
  +--> ?PR?_LCDDISPSTRING?TFTLCD
  +--> ?PR?RESSTART?GAME
  +--> ?PR?RETRACTCHESS?GAME

?PR?_CLEARSELECTBOX?GAME             1DC1H    0004H
  +--> ?PR?_LCDSETCOLOR?TFTLCD
  +--> ?PR?_LCDDRAWRECT?TFTLCD

?PR?_DRAWCHESS?GAME                  1DC1H    0004H
  +--> ?PR?_LCDDRAWCIRCLEA?TFTLCD

?PR?_LCDDRAWCIRCLEA?TFTLCD           1DCDH    0011H
  +--> ?PR?_LCDDRAWLINE?TFTLCD
  +--> ?PR?_LCDDRAWPOINT?TFTLCD

?PR?_ISGAMEOVER?GAME                 -----    -----
  +--> ?PR?_ISFIVECHESSCONTANT?GAME

?PR?_ISFIVECHESSCONTANT?GAME         1DC1H    0006H
  +--> ?PR?_GETCHESSNUM?GAME

?PR?_GETCHESSNUM?GAME                1DC7H    0009H

?PR?_LCDDISPSTRING?TFTLCD            1DC1H    0011H
  +--> ?PR?_LCDDISPCHAR?TFTLCD

?PR?_LCDDISPCHAR?TFTLCD              1DD2H    000CH
  +--> ?CO?TFTLCD
  +--> ?PR?_LCDDRAWPOINT?TFTLCD

?PR?RESSTART?GAME                    1DC1H    0004H
  +--> ?PR?DRAWCHESSBOARD?GAME
  +--> ?PR?_DRAWSELECTBOX?GAME

?PR?RETRACTCHESS?GAME                1DC1H    0008H
  +--> ?PR?_CLEARCHESS?GAME

?PR?_CLEARCHESS?GAME                 1DC9H    0004H
BL51 BANKED LINKER/LOCATER V6.22                                                      11/30/2016  13:53:19  PAGE 5


  +--> ?PR?_LCDDRAWCIRCLEA?TFTLCD

?C_INITSEG                           -----    -----
  +--> ?PR?_MEM_INIT?MALLOC
  +--> ?PR?_MEM_PERUSED?MALLOC

?PR?_MEM_INIT?MALLOC                 1DC0H    0001H
  +--> ?PR?_MYMEMSET?MALLOC

?PR?_MYMEMSET?MALLOC                 1DC1H    000BH

?PR?_MEM_PERUSED?MALLOC              1DC0H    0009H



SYMBOL TABLE OF MODULE:  .\Objects\RAM (?C_STARTUP)

  VALUE           TYPE          NAME
  ----------------------------------

  -------         MODULE        ?C_STARTUP
  C:403BH         SEGMENT       ?C_C51STARTUP
  I:0022H         SEGMENT       ?STACK
  C:0000H         PUBLIC        ?C_STARTUP
  D:00E0H         SYMBOL        ACC
  D:00F0H         SYMBOL        B
  D:0083H         SYMBOL        DPH
  D:0082H         SYMBOL        DPL
  N:0000H         SYMBOL        IBPSTACK
  N:0100H         SYMBOL        IBPSTACKTOP
  N:0080H         SYMBOL        IDATALEN
  C:403EH         SYMBOL        IDATALOOP
  N:0000H         SYMBOL        PBPSTACK
  N:0100H         SYMBOL        PBPSTACKTOP
  N:0000H         SYMBOL        PDATALEN
  N:0000H         SYMBOL        PDATASTART
  N:0000H         SYMBOL        PPAGE
  N:0000H         SYMBOL        PPAGEENABLE
  D:00A0H         SYMBOL        PPAGE_SFR
  D:0081H         SYMBOL        SP
  C:403BH         SYMBOL        STARTUP1
  N:0000H         SYMBOL        XBPSTACK
  N:0000H         SYMBOL        XBPSTACKTOP
  N:0000H         SYMBOL        XDATALEN
  N:0000H         SYMBOL        XDATASTART
  C:0000H         LINE#         126
  C:403BH         LINE#         133
  C:403DH         LINE#         134
  C:403EH         LINE#         135
  C:403FH         LINE#         136
  C:4041H         LINE#         185
  C:4044H         LINE#         196
  -------         ENDMOD        ?C_STARTUP

  -------         MODULE        MAIN
  C:0000H         SYMBOL        _ICE_DUMMY_
  D:00B0H         PUBLIC        P3
BL51 BANKED LINKER/LOCATER V6.22                                                      11/30/2016  13:53:19  PAGE 6


  C:45EFH         PUBLIC        main
  -------         PROC          MAIN
  C:45EFH         LINE#         6
  C:45EFH         LINE#         7
  C:45EFH         LINE#         9
  C:4600H         LINE#         11
  C:4603H         LINE#         13
  C:4603H         LINE#         14
  C:4603H         LINE#         16
  C:4606H         LINE#         17
  -------         ENDPROC       MAIN
  -------         ENDMOD        MAIN

  -------         MODULE        GAME
  C:0000H         SYMBOL        _ICE_DUMMY_
  D:00B0H         PUBLIC        P3
  C:3BCDH         SYMBOL        _DrawChess
  C:2951H         PUBLIC        GameStart
  C:44EDH         PUBLIC        GameInit
  C:2FF9H         SYMBOL        _IsFiveChessContant
  C:42A1H         SYMBOL        _DrawSelectBox
  C:40C7H         SYMBOL        ResStart
  X:1EA4H         PUBLIC        g_Chess
  C:31D3H         SYMBOL        _GetChessNum
  C:39E1H         SYMBOL        RetractChess
  C:45B3H         SYMBOL        _IsGameOver
  C:3FA8H         SYMBOL        _ClearChess
  X:1EA7H         PUBLIC        g_ChessNum
  C:37CBH         SYMBOL        DrawChessBoard
  C:4243H         SYMBOL        _ClearSelectBox
  X:1EA9H         PUBLIC        g_SameChessNum
  -------         PROC          DRAWCHESSBOARD
  -------         DO            
  X:1DC5H         SYMBOL        i
  -------         ENDDO         
  C:37CBH         LINE#         24
  C:37CBH         LINE#         25
  C:37CBH         LINE#         28
  C:37E9H         LINE#         30
  C:37EFH         LINE#         32
  C:3807H         LINE#         34
  C:381FH         LINE#         36
  C:3837H         LINE#         40
  C:3851H         LINE#         41
  C:3851H         LINE#         42
  C:3875H         LINE#         47
  C:3885H         LINE#         50
  C:389FH         LINE#         51
  C:389FH         LINE#         52
  C:38CCH         LINE#         57
  C:38DCH         LINE#         58
  -------         ENDPROC       DRAWCHESSBOARD
  -------         PROC          _DRAWCHESS
  X:1DC1H         SYMBOL        x
  X:1DC2H         SYMBOL        y
  -------         DO            
  X:1DC3H         SYMBOL        ChessColor
BL51 BANKED LINKER/LOCATER V6.22                                                      11/30/2016  13:53:19  PAGE 7


  D:0004H         SYMBOL        xChess
  D:0002H         SYMBOL        yChess
  -------         ENDDO         
  C:3BCDH         LINE#         62
  C:3BD7H         LINE#         63
  C:3BD7H         LINE#         68
  C:3BFDH         LINE#         69
  C:3C26H         LINE#         72
  C:3C43H         LINE#         75
  C:3C54H         LINE#         76
  C:3C62H         LINE#         78
  C:3C81H         LINE#         83
  C:3C8FH         LINE#         84
  C:3CBDH         LINE#         85
  -------         ENDPROC       _DRAWCHESS
  -------         PROC          _CLEARCHESS
  X:1DC9H         SYMBOL        x
  X:1DCAH         SYMBOL        y
  -------         DO            
  X:1DCBH         SYMBOL        ChessColor
  D:0004H         SYMBOL        xChess
  D:0002H         SYMBOL        yChess
  -------         ENDDO         
  C:3FA8H         LINE#         89
  C:3FB2H         LINE#         90
  C:3FB2H         LINE#         95
  C:3FCFH         LINE#         96
  C:3FF5H         LINE#         98
  C:3FFFH         LINE#         101
  C:4010H         LINE#         102
  C:401EH         LINE#         104
  C:403AH         LINE#         109
  -------         ENDPROC       _CLEARCHESS
  -------         PROC          _DRAWSELECTBOX
  D:0007H         SYMBOL        x
  D:0005H         SYMBOL        y
  -------         DO            
  X:1DC5H         SYMBOL        xChess
  X:1DC7H         SYMBOL        yChess
  -------         ENDDO         
  C:42A1H         LINE#         113
  C:42A1H         LINE#         114
  C:42A1H         LINE#         117
  C:42B3H         LINE#         118
  C:42C3H         LINE#         120
  C:42CAH         LINE#         122
  -------         ENDPROC       _DRAWSELECTBOX
  C:4239H         SYMBOL        L?0151
  -------         PROC          L?0150
  -------         ENDPROC       L?0150
  C:4239H         SYMBOL        L?0151
  -------         PROC          _CLEARSELECTBOX
  D:0007H         SYMBOL        x
  D:0005H         SYMBOL        y
  -------         DO            
  X:1DC1H         SYMBOL        xChess
  X:1DC3H         SYMBOL        yChess
BL51 BANKED LINKER/LOCATER V6.22                                                      11/30/2016  13:53:19  PAGE 8


  -------         ENDDO         
  C:4243H         LINE#         130
  C:4243H         LINE#         131
  C:4243H         LINE#         134
  C:4255H         LINE#         135
  C:4265H         LINE#         137
  C:426BH         LINE#         138
  -------         ENDPROC       _CLEARSELECTBOX
  C:31CFH         SYMBOL        L?0153
  -------         PROC          L?0152
  -------         ENDPROC       L?0152
  C:31CFH         SYMBOL        L?0153
  -------         PROC          _GETCHESSNUM
  X:1DC7H         SYMBOL        ChessType
  X:1DC8H         SYMBOL        x
  X:1DCAH         SYMBOL        y
  X:1DCCH         SYMBOL        xStep
  X:1DCEH         SYMBOL        yStep
  C:31D3H         LINE#         147
  C:31E4H         LINE#         148
  C:31E4H         LINE#         149
  C:31EBH         LINE#         150
  C:31EBH         LINE#         151
  C:31EBH         LINE#         152
  C:31FFH         LINE#         153
  C:3213H         LINE#         156
  C:3247H         LINE#         157
  C:3247H         LINE#         158
  C:324AH         LINE#         159
  C:324AH         LINE#         162
  C:327AH         LINE#         163
  C:327AH         LINE#         164
  C:327DH         LINE#         165
  C:327DH         LINE#         168
  C:3290H         LINE#         169
  C:3290H         LINE#         170
  C:32B5H         LINE#         171
  C:32B5H         LINE#         172
  C:32C3H         LINE#         173
  C:32C6H         LINE#         174
  C:32F1H         LINE#         175
  C:32F1H         LINE#         176
  C:32FFH         LINE#         177
  C:3302H         LINE#         178
  C:332AH         LINE#         179
  C:332AH         LINE#         180
  C:3338H         LINE#         181
  C:333BH         LINE#         182
  C:336CH         LINE#         183
  C:336CH         LINE#         184
  C:337AH         LINE#         185
  C:337AH         LINE#         186
  C:337DH         LINE#         188
  C:337DH         LINE#         189
  C:3385H         LINE#         190
  C:3385H         LINE#         191
  C:3385H         LINE#         192
BL51 BANKED LINKER/LOCATER V6.22                                                      11/30/2016  13:53:19  PAGE 9


  -------         ENDPROC       _GETCHESSNUM
  -------         PROC          _ISFIVECHESSCONTANT
  X:1DC1H         SYMBOL        x
  X:1DC3H         SYMBOL        y
  -------         DO            
  X:1DC5H         SYMBOL        ChessType
  D:0004H         SYMBOL        ChessNum
  -------         ENDDO         
  C:2FF9H         LINE#         196
  C:3009H         LINE#         197
  C:3009H         LINE#         198
  C:3010H         LINE#         199
  C:3011H         LINE#         201
  C:3048H         LINE#         204
  C:3094H         LINE#         206
  C:309FH         LINE#         207
  C:309FH         LINE#         208
  C:30A2H         LINE#         209
  C:30A2H         LINE#         212
  C:30F4H         LINE#         214
  C:30FFH         LINE#         215
  C:30FFH         LINE#         216
  C:3102H         LINE#         217
  C:3102H         LINE#         220
  C:3157H         LINE#         222
  C:3162H         LINE#         223
  C:3162H         LINE#         224
  C:3165H         LINE#         225
  C:3165H         LINE#         228
  C:31BAH         LINE#         230
  C:31C6H         LINE#         231
  C:31C6H         LINE#         232
  C:31C9H         LINE#         233
  C:31C9H         LINE#         235
  C:31CBH         LINE#         236
  -------         ENDPROC       _ISFIVECHESSCONTANT
  -------         PROC          _ISGAMEOVER
  D:0007H         SYMBOL        x
  D:0005H         SYMBOL        y
  C:45B3H         LINE#         242
  C:45B3H         LINE#         243
  C:45B3H         LINE#         245
  C:45C0H         LINE#         248
  C:45CFH         LINE#         250
  C:45D1H         LINE#         251
  -------         ENDPROC       _ISGAMEOVER
  -------         PROC          RETRACTCHESS
  -------         DO            
  X:1DC1H         SYMBOL        x
  X:1DC3H         SYMBOL        y
  X:1DC5H         SYMBOL        xChess
  X:1DC7H         SYMBOL        yChess
  -------         ENDDO         
  C:39E1H         LINE#         254
  C:39E1H         LINE#         255
  C:39E1H         LINE#         260
  C:39EEH         LINE#         263
BL51 BANKED LINKER/LOCATER V6.22                                                      11/30/2016  13:53:19  PAGE 10


  C:39F5H         LINE#         264
  C:39F5H         LINE#         265
  C:39FCH         LINE#         266
  C:39FCH         LINE#         267
  C:3A3AH         LINE#         268
  C:3A3AH         LINE#         269
  C:3A49H         LINE#         270
  C:3A58H         LINE#         271
  C:3A5AH         LINE#         272
  C:3A5AH         LINE#         273
  C:3A74H         LINE#         274
  C:3A91H         LINE#         277
  C:3AC0H         LINE#         278
  C:3ACEH         LINE#         279
  C:3AD7H         LINE#         280
  -------         ENDPROC       RETRACTCHESS
  -------         PROC          RESSTART
  -------         DO            
  X:1DC1H         SYMBOL        xChess
  X:1DC3H         SYMBOL        yChess
  -------         ENDDO         
  C:40C7H         LINE#         283
  C:40C7H         LINE#         284
  C:40C7H         LINE#         287
  C:40CEH         LINE#         289
  C:40D4H         LINE#         290
  C:40D4H         LINE#         291
  C:40DBH         LINE#         292
  C:40DBH         LINE#         293
  C:4109H         LINE#         294
  C:4123H         LINE#         295
  C:413DH         LINE#         297
  C:4140H         LINE#         299
  -------         ENDPROC       RESSTART
  -------         PROC          GAMEINIT
  C:44EDH         LINE#         305
  C:44EDH         LINE#         306
  C:44EDH         LINE#         307
  C:44F4H         LINE#         308
  C:450EH         LINE#         309
  C:4514H         LINE#         311
  C:4517H         LINE#         313
  -------         ENDPROC       GAMEINIT
  -------         PROC          GAMESTART
  -------         DO            
  X:1EA0H         SYMBOL        xChess
  X:1EA2H         SYMBOL        yChess
  D:0007H         SYMBOL        key
  X:1DC0H         SYMBOL        State
  -------         ENDDO         
  C:2951H         LINE#         317
  C:2951H         LINE#         318
  C:2951H         LINE#         325
  C:2954H         LINE#         327
  C:297FH         LINE#         328
  C:297FH         LINE#         329
  C:297FH         LINE#         330
BL51 BANKED LINKER/LOCATER V6.22                                                      11/30/2016  13:53:19  PAGE 11


  C:2987H         LINE#         331
  C:298AH         LINE#         332
  C:2998H         LINE#         333
  C:29A6H         LINE#         334
  C:29A6H         LINE#         335
  C:29A9H         LINE#         336
  C:29A9H         LINE#         337
  C:29B1H         LINE#         338
  C:29B4H         LINE#         339
  C:29C2H         LINE#         340
  C:29D0H         LINE#         341
  C:29D0H         LINE#         342
  C:29D2H         LINE#         343
  C:29D2H         LINE#         344
  C:29DAH         LINE#         345
  C:29DDH         LINE#         346
  C:29EBH         LINE#         347
  C:2A00H         LINE#         348
  C:2A00H         LINE#         349
  C:2A02H         LINE#         350
  C:2A02H         LINE#         351
  C:2A0AH         LINE#         352
  C:2A0DH         LINE#         353
  C:2A1BH         LINE#         354
  C:2A30H         LINE#         355
  C:2A3DH         LINE#         356
  C:2A3DH         LINE#         357
  C:2A3DH         LINE#         358
  C:2A45H         LINE#         359
  C:2A52H         LINE#         360
  C:2A64H         LINE#         361
  C:2A6DH         LINE#         362
  C:2A6DH         LINE#         363
  C:2A74H         LINE#         364
  C:2A82H         LINE#         365
  C:2A82H         LINE#         366
  C:2A82H         LINE#         367
  C:2AA0H         LINE#         368
  C:2ACBH         LINE#         369
  C:2ACBH         LINE#         370
  C:2ACEH         LINE#         371
  C:2ACEH         LINE#         372
  C:2AECH         LINE#         373
  C:2B28H         LINE#         374
  C:2B28H         LINE#         375
  C:2B39H         LINE#         376
  C:2B3BH         LINE#         378
  C:2B3BH         LINE#         379
  C:2B63H         LINE#         380
  C:2B63H         LINE#         381
  C:2B69H         LINE#         382
  C:2B69H         LINE#         383
  C:2B69H         LINE#         384
  C:2B69H         LINE#         385
  C:2B69H         LINE#         386
  C:2B6FH         LINE#         388
  C:2B7AH         LINE#         389
BL51 BANKED LINKER/LOCATER V6.22                                                      11/30/2016  13:53:19  PAGE 12


  C:2B7AH         LINE#         390
  C:2B82H         LINE#         391
  C:2B82H         LINE#         392
  C:2B82H         LINE#         393
  C:2B82H         LINE#         394
  C:2B84H         LINE#         395
  C:2B84H         LINE#         396
  C:2B84H         LINE#         397
  C:2B84H         LINE#         398
  C:2B84H         LINE#         399
  C:2B8CH         LINE#         400
  C:2B8FH         LINE#         401
  C:2B98H         LINE#         402
  C:2B9FH         LINE#         403
  C:2BA0H         LINE#         404
  C:2BA0H         LINE#         405
  C:2BA8H         LINE#         406
  C:2BABH         LINE#         407
  C:2BABH         LINE#         408
  C:2BABH         LINE#         409
  C:2BABH         LINE#         410
  C:2BABH         LINE#         411
  -------         ENDPROC       GAMESTART
  -------         ENDMOD        GAME

  -------         MODULE        MALLOC
  C:0000H         SYMBOL        _ICE_DUMMY_
  X:1E57H         PUBLIC        memsize
  C:4147H         PUBLIC        _myfree
  X:0000H         PUBLIC        mem2base
  C:26ECH         PUBLIC        _mem_malloc
  X:1E5BH         PUBLIC        mallco_dev
  C:3AD8H         PUBLIC        _mem_perused
  X:1E68H         PUBLIC        memblksize
  X:1E6CH         PUBLIC        memtblsize
  C:3699H         PUBLIC        _mem_free
  C:38DDH         PUBLIC        _myrealloc
  X:1C00H         PUBLIC        mem2mapbase
  C:3E6CH         PUBLIC        _mem_init
  C:41C0H         PUBLIC        _mymalloc
  C:4300H         PUBLIC        _mymemcpy
  C:447EH         PUBLIC        _mymemset
  -------         PROC          _MYMEMCPY
  D:0001H         SYMBOL        des
  X:1E87H         SYMBOL        src
  X:1E8AH         SYMBOL        n
  -------         DO            
  X:1E8EH         SYMBOL        xdes
  X:1E91H         SYMBOL        xsrc
  -------         ENDDO         
  C:4300H         LINE#         26
  C:4300H         LINE#         27
  C:4300H         LINE#         28
  C:430BH         LINE#         29
  C:4320H         LINE#         30
  C:4358H         LINE#         31
  -------         ENDPROC       _MYMEMCPY
BL51 BANKED LINKER/LOCATER V6.22                                                      11/30/2016  13:53:19  PAGE 13


  -------         PROC          _MYMEMSET
  D:0001H         SYMBOL        s
  X:1DC4H         SYMBOL        c
  X:1DC5H         SYMBOL        count
  -------         DO            
  X:1DC9H         SYMBOL        xs
  -------         ENDDO         
  C:447EH         LINE#         37
  C:4483H         LINE#         38
  C:4483H         LINE#         39
  C:448EH         LINE#         40
  C:44B7H         LINE#         41
  -------         ENDPROC       _MYMEMSET
  -------         PROC          _MEM_INIT
  X:1DC0H         SYMBOL        memx
  C:3E6CH         LINE#         45
  C:3E71H         LINE#         46
  C:3E71H         LINE#         47
  C:3EC1H         LINE#         48
  C:3EFFH         LINE#         49
  C:3F0FH         LINE#         50
  -------         ENDPROC       _MEM_INIT
  -------         PROC          _MEM_PERUSED
  X:1DC0H         SYMBOL        memx
  -------         DO            
  X:1DC1H         SYMBOL        used
  X:1DC5H         SYMBOL        i
  -------         ENDDO         
  C:3AD8H         LINE#         55
  C:3ADDH         LINE#         56
  C:3ADDH         LINE#         57
  C:3AE5H         LINE#         59
  C:3B1FH         LINE#         60
  C:3B1FH         LINE#         61
  C:3B74H         LINE#         62
  C:3B96H         LINE#         63
  C:3BCCH         LINE#         64
  -------         ENDPROC       _MEM_PERUSED
  -------         PROC          _MEM_MALLOC
  X:1DC9H         SYMBOL        memx
  X:1DCAH         SYMBOL        nsize
  -------         DO            
  X:1DCEH         SYMBOL        offset
  X:1DD2H         SYMBOL        nmemb
  X:1DD4H         SYMBOL        cmemb
  X:1DD6H         SYMBOL        i
  -------         ENDDO         
  C:26ECH         LINE#         70
  C:26F1H         LINE#         71
  C:26F1H         LINE#         72
  C:26FBH         LINE#         74
  C:2702H         LINE#         76
  C:2722H         LINE#         77
  C:273EH         LINE#         78
  C:2773H         LINE#         79
  C:27BCH         LINE#         80
  C:27E6H         LINE#         81
BL51 BANKED LINKER/LOCATER V6.22                                                      11/30/2016  13:53:19  PAGE 14


  C:27E6H         LINE#         82
  C:2831H         LINE#         83
  C:2838H         LINE#         84
  C:284DH         LINE#         85
  C:284DH         LINE#         86
  C:2879H         LINE#         87
  C:2879H         LINE#         88
  C:28D4H         LINE#         89
  C:28F6H         LINE#         90
  C:2923H         LINE#         91
  C:2923H         LINE#         92
  C:294AH         LINE#         93
  C:2950H         LINE#         94
  -------         ENDPROC       _MEM_MALLOC
  -------         PROC          _MEM_FREE
  X:1EABH         SYMBOL        memx
  X:1EACH         SYMBOL        offset
  -------         DO            
  X:1EB0H         SYMBOL        i
  -------         DO            
  X:1EB2H         SYMBOL        index
  X:1EB4H         SYMBOL        nmemb
  -------         ENDDO         
  -------         ENDDO         
  C:3699H         LINE#         100
  C:369EH         LINE#         101
  C:369EH         LINE#         103
  C:36ACH         LINE#         104
  C:36ACH         LINE#         105
  C:36BBH         LINE#         106
  C:36BEH         LINE#         107
  C:36BEH         LINE#         108
  C:36F1H         LINE#         109
  C:36F1H         LINE#         110
  C:3726H         LINE#         111
  C:375CH         LINE#         112
  C:377FH         LINE#         113
  C:377FH         LINE#         114
  C:37B5H         LINE#         115
  C:37C5H         LINE#         116
  C:37C8H         LINE#         117
  C:37CAH         LINE#         118
  -------         ENDPROC       _MEM_FREE
  -------         PROC          _MYFREE
  X:1EC0H         SYMBOL        memx
  X:1EC1H         SYMBOL        ptr
  -------         DO            
  X:1EC4H         SYMBOL        offset
  -------         ENDDO         
  C:4147H         LINE#         123
  C:4155H         LINE#         124
  C:4155H         LINE#         126
  C:4158H         LINE#         127
  C:41A3H         LINE#         128
  C:41BFH         LINE#         129
  -------         ENDPROC       _MYFREE
  -------         PROC          _MYMALLOC
BL51 BANKED LINKER/LOCATER V6.22                                                      11/30/2016  13:53:19  PAGE 15


  X:1DC0H         SYMBOL        memx
  X:1DC1H         SYMBOL        nsize
  -------         DO            
  X:1DC5H         SYMBOL        offset
  -------         ENDDO         
  C:41C0H         LINE#         135
  C:41C5H         LINE#         136
  C:41C5H         LINE#         138
  C:41E4H         LINE#         139
  C:4202H         LINE#         140
  C:4238H         LINE#         141
  -------         ENDPROC       _MYMALLOC
  -------         PROC          _MYREALLOC
  X:1E94H         SYMBOL        memx
  X:1E95H         SYMBOL        ptr
  X:1E98H         SYMBOL        nsize
  -------         DO            
  X:1E9CH         SYMBOL        offset
  -------         ENDDO         
  C:38DDH         LINE#         148
  C:38EBH         LINE#         149
  C:38EBH         LINE#         151
  C:390BH         LINE#         152
  C:3929H         LINE#         154
  C:3929H         LINE#         155
  C:3999H         LINE#         156
  C:39AAH         LINE#         157
  C:39E0H         LINE#         158
  C:39E0H         LINE#         159
  -------         ENDPROC       _MYREALLOC
  -------         ENDMOD        MALLOC

  -------         MODULE        TFTLCD
  C:0000H         SYMBOL        _ICE_DUMMY_
  C:4359H         PUBLIC        _LcdClear
  D:0090H         PUBLIC        P1
  D:00B0H         PUBLIC        P3
  C:4593H         PUBLIC        LcdReadData
  C:0A67H         PUBLIC        asc2_2412
  C:0003H         PUBLIC        asc2_1206
  C:0477H         PUBLIC        asc2_1608
  C:3F10H         PUBLIC        _LcdFill
  C:461EH         PUBLIC        _LcdWriteData
  C:3386H         PUBLIC        _LcdDispString
  C:353AH         PUBLIC        _LcdDispChar
  X:1E70H         PUBLIC        lcd_printf
  C:2E0BH         PUBLIC        _LcdDrawLine
  C:445DH         PUBLIC        _LcdDrawPoint
  C:3CBEH         PUBLIC        _LcdDrawRect
  C:17C3H         PUBLIC        _LcdDrawCircleA
  C:460EH         PUBLIC        _LcdWriteCom
  C:4645H         PUBLIC        _LcdSetColor
  C:3D9FH         PUBLIC        _LCD_printf
  C:45D2H         PUBLIC        _delay_ms
  B:00B0H.2       PUBLIC        LCD_RS
  C:462EH         PUBLIC        _delay_us
  B:00B0H.1       PUBLIC        LCD_RW
BL51 BANKED LINKER/LOCATER V6.22                                                      11/30/2016  13:53:19  PAGE 16


  C:463CH         PUBLIC        _LcdSetBkColor
  X:1E7CH         PUBLIC        lcddev
  C:451EH         PUBLIC        _LcdSetPos
  B:00B0H.0       PUBLIC        LCD_E
  C:2BACH         PUBLIC        _LcdDrawCircle
  -------         PROC          _DELAY_US
  D:0006H         SYMBOL        us
  C:462EH         LINE#         30
  C:462EH         LINE#         31
  C:462EH         LINE#         32
  C:4638H         LINE#         33
  C:4638H         LINE#         34
  C:4639H         LINE#         35
  C:463BH         LINE#         36
  -------         ENDPROC       _DELAY_US
  -------         PROC          _DELAY_MS
  D:0006H         SYMBOL        ms
  -------         DO            
  D:0005H         SYMBOL        i
  D:0004H         SYMBOL        j
  -------         ENDDO         
  C:45D2H         LINE#         40
  C:45D2H         LINE#         41
  C:45D2H         LINE#         43
  C:45DCH         LINE#         44
  C:45DCH         LINE#         45
  C:45E4H         LINE#         46
  C:45EEH         LINE#         47
  C:45EEH         LINE#         48
  -------         ENDPROC       _DELAY_MS
  C:4609H         SYMBOL        L?0148
  -------         PROC          L?0147
  -------         ENDPROC       L?0147
  C:4609H         SYMBOL        L?0148
  -------         PROC          _LCDWRITECOM
  D:0007H         SYMBOL        com
  C:460EH         LINE#         52
  C:460EH         LINE#         53
  C:460EH         LINE#         54
  C:4610H         LINE#         55
  C:4612H         LINE#         56
  C:4614H         LINE#         57
  C:4617H         LINE#         58
  C:4619H         LINE#         59
  C:461BH         LINE#         60
  C:461DH         LINE#         61
  -------         ENDPROC       _LCDWRITECOM
  -------         PROC          _LCDWRITEDATA
  D:0007H         SYMBOL        dat
  C:461EH         LINE#         65
  C:461EH         LINE#         66
  C:461EH         LINE#         67
  C:4620H         LINE#         68
  C:4622H         LINE#         69
  C:4624H         LINE#         70
  C:4627H         LINE#         71
  C:4629H         LINE#         72
BL51 BANKED LINKER/LOCATER V6.22                                                      11/30/2016  13:53:19  PAGE 17


  C:462BH         LINE#         73
  C:462DH         LINE#         74
  -------         ENDPROC       _LCDWRITEDATA
  -------         PROC          LCDREADDATA
  -------         DO            
  D:0006H         SYMBOL        dat
  -------         ENDDO         
  C:4593H         LINE#         77
  C:4593H         LINE#         78
  C:4593H         LINE#         80
  C:4596H         LINE#         81
  C:4598H         LINE#         82
  C:459AH         LINE#         83
  C:459CH         LINE#         84
  C:45A3H         LINE#         85
  C:45A5H         LINE#         86
  C:45ACH         LINE#         87
  C:45B0H         LINE#         88
  C:45B2H         LINE#         89
  C:45B2H         LINE#         90
  -------         ENDPROC       LCDREADDATA
  C:4442H         SYMBOL        L?0139
  C:4443H         SYMBOL        L?0140
  C:4454H         SYMBOL        L?0141
  C:4455H         SYMBOL        L?0142
  C:4458H         SYMBOL        L?0143
  -------         PROC          L?0138
  -------         ENDPROC       L?0138
  C:4442H         SYMBOL        L?0139
  C:4443H         SYMBOL        L?0140
  C:4454H         SYMBOL        L?0141
  C:4455H         SYMBOL        L?0142
  C:4458H         SYMBOL        L?0143
  -------         PROC          _LCDDRAWPOINT
  X:1DFCH         SYMBOL        x
  D:0004H         SYMBOL        y
  D:0002H         SYMBOL        color
  C:445DH         LINE#         95
  C:4465H         LINE#         96
  C:4465H         LINE#         97
  C:4468H         LINE#         98
  C:446CH         LINE#         99
  C:446FH         LINE#         100
  C:4474H         LINE#         101
  C:4479H         LINE#         102
  -------         ENDPROC       _LCDDRAWPOINT
  C:2DF0H         SYMBOL        L?0145
  C:2E06H         SYMBOL        L?0146
  -------         PROC          L?0144
  -------         ENDPROC       L?0144
  C:2DF0H         SYMBOL        L?0145
  C:2E06H         SYMBOL        L?0146
  -------         PROC          _LCDDRAWLINE
  X:1DDEH         SYMBOL        x0
  X:1DE0H         SYMBOL        y0
  D:0002H         SYMBOL        x1
  X:1DE4H         SYMBOL        y1
BL51 BANKED LINKER/LOCATER V6.22                                                      11/30/2016  13:53:19  PAGE 18


  X:1DE6H         SYMBOL        color
  -------         DO            
  X:1DE8H         SYMBOL        t
  X:1DEAH         SYMBOL        xerr
  X:1DECH         SYMBOL        yerr
  X:1DEEH         SYMBOL        delta_x
  X:1DF0H         SYMBOL        delta_y
  X:1DF2H         SYMBOL        distance
  X:1DF4H         SYMBOL        incx
  X:1DF6H         SYMBOL        incy
  X:1DF8H         SYMBOL        uRow
  X:1DFAH         SYMBOL        uCol
  -------         ENDDO         
  C:2E0BH         LINE#         109
  C:2E19H         LINE#         110
  C:2E19H         LINE#         112
  C:2E24H         LINE#         114
  C:2E39H         LINE#         115
  C:2E54H         LINE#         116
  C:2E63H         LINE#         117
  C:2E69H         LINE#         118
  C:2E85H         LINE#         119
  C:2E91H         LINE#         120
  C:2EA6H         LINE#         121
  C:2EC2H         LINE#         122
  C:2ECEH         LINE#         123
  C:2EE3H         LINE#         124
  C:2F09H         LINE#         125
  C:2F0EH         LINE#         127
  C:2F33H         LINE#         128
  C:2F33H         LINE#         129
  C:2F47H         LINE#         130
  C:2F5BH         LINE#         131
  C:2F6FH         LINE#         132
  C:2F8BH         LINE#         133
  C:2F8BH         LINE#         134
  C:2F97H         LINE#         135
  C:2FABH         LINE#         136
  C:2FABH         LINE#         137
  C:2FC7H         LINE#         138
  C:2FC7H         LINE#         139
  C:2FD3H         LINE#         140
  C:2FE7H         LINE#         141
  C:2FE7H         LINE#         142
  C:2FF8H         LINE#         143
  -------         ENDPROC       _LCDDRAWLINE
  -------         PROC          _LCDDRAWRECT
  X:1DC9H         SYMBOL        x1
  X:1DCBH         SYMBOL        y1
  X:1DCDH         SYMBOL        x2
  X:1DCFH         SYMBOL        y2
  C:3CBEH         LINE#         148
  C:3CD4H         LINE#         149
  C:3CD4H         LINE#         150
  C:3CFFH         LINE#         151
  C:3D35H         LINE#         152
  C:3D67H         LINE#         153
BL51 BANKED LINKER/LOCATER V6.22                                                      11/30/2016  13:53:19  PAGE 19


  -------         ENDPROC       _LCDDRAWRECT
  -------         PROC          _LCDDRAWCIRCLE
  X:1EB6H         SYMBOL        x0
  X:1EB8H         SYMBOL        y0
  D:0003H         SYMBOL        r
  -------         DO            
  X:1EBAH         SYMBOL        a
  X:1EBCH         SYMBOL        b
  X:1EBEH         SYMBOL        di
  -------         ENDDO         
  C:2BACH         LINE#         159
  C:2BBAH         LINE#         160
  C:2BBAH         LINE#         163
  C:2BC9H         LINE#         164
  C:2BDDH         LINE#         165
  C:2BFCH         LINE#         166
  C:2BFCH         LINE#         167
  C:2C23H         LINE#         168
  C:2C52H         LINE#         169
  C:2C80H         LINE#         170
  C:2CAEH         LINE#         171
  C:2CDDH         LINE#         172
  C:2D0CH         LINE#         173
  C:2D3CH         LINE#         174
  C:2D6CH         LINE#         175
  C:2D7AH         LINE#         177
  C:2DAAH         LINE#         179
  C:2DAAH         LINE#         180
  C:2DDBH         LINE#         181
  C:2DE9H         LINE#         182
  C:2DE9H         LINE#         183
  C:2DECH         LINE#         184
  -------         ENDPROC       _LCDDRAWCIRCLE
  -------         PROC          _LCDDRAWCIRCLEA
  X:1DCDH         SYMBOL        x
  X:1DCFH         SYMBOL        y
  X:1DD1H         SYMBOL        r
  X:1DD3H         SYMBOL        color
  X:1DD5H         SYMBOL        Mode
  -------         DO            
  X:1DD6H         SYMBOL        dx
  X:1DD8H         SYMBOL        dy
  X:1DDAH         SYMBOL        ref
  X:1DDCH         SYMBOL        Temp
  -------         ENDDO         
  C:17C3H         LINE#         187
  C:17D7H         LINE#         188
  C:17D7H         LINE#         192
  C:17DDH         LINE#         194
  C:17EDH         LINE#         195
  C:17F3H         LINE#         196
  C:1806H         LINE#         198
  C:1811H         LINE#         199
  C:1811H         LINE#         200
  C:182FH         LINE#         201
  C:182FH         LINE#         202
  C:1843H         LINE#         203
BL51 BANKED LINKER/LOCATER V6.22                                                      11/30/2016  13:53:19  PAGE 20


  C:18B1H         LINE#         205
  C:18E8H         LINE#         206
  C:18E8H         LINE#         207
  C:1900H         LINE#         208
  C:1909H         LINE#         210
  C:1916H         LINE#         211
  C:195CH         LINE#         212
  C:195CH         LINE#         214
  C:1996H         LINE#         215
  C:1A00H         LINE#         216
  C:1A54H         LINE#         217
  C:1A54H         LINE#         218
  C:1A6CH         LINE#         219
  C:1A75H         LINE#         221
  C:1A82H         LINE#         222
  C:1ACAH         LINE#         223
  C:1ACAH         LINE#         225
  C:1AEDH         LINE#         226
  C:1AEDH         LINE#         227
  C:1B09H         LINE#         228
  C:1B12H         LINE#         230
  C:1B1FH         LINE#         231
  C:1B72H         LINE#         232
  C:1B72H         LINE#         234
  C:1BB7H         LINE#         235
  C:1BB7H         LINE#         236
  C:1BD3H         LINE#         237
  C:1BDCH         LINE#         239
  C:1BE9H         LINE#         240
  C:1C3DH         LINE#         241
  C:1C3DH         LINE#         242
  C:1C4BH         LINE#         243
  C:1C94H         LINE#         244
  C:1C9FH         LINE#         245
  C:1CA2H         LINE#         247
  C:1CFDH         LINE#         249
  C:1D1FH         LINE#         250
  C:1D1FH         LINE#         251
  C:1D33H         LINE#         252
  C:1D3CH         LINE#         254
  C:1D49H         LINE#         255
  C:1D79H         LINE#         256
  C:1D79H         LINE#         258
  C:1D95H         LINE#         259
  C:1D9EH         LINE#         261
  C:1DABH         LINE#         262
  C:1DF2H         LINE#         263
  C:1DF2H         LINE#         265
  C:1DF2H         LINE#         266
  C:1E10H         LINE#         267
  C:1E10H         LINE#         268
  C:1E32H         LINE#         269
  C:1E5DH         LINE#         270
  C:1E73H         LINE#         271
  C:1E8AH         LINE#         272
  C:1EA1H         LINE#         273
  C:1EA1H         LINE#         274
BL51 BANKED LINKER/LOCATER V6.22                                                      11/30/2016  13:53:19  PAGE 21


  C:1EC3H         LINE#         275
  C:1EDCH         LINE#         276
  C:1F07H         LINE#         277
  C:1F22H         LINE#         278
  C:1F22H         LINE#         279
  C:1F30H         LINE#         280
  C:1F79H         LINE#         281
  C:1F84H         LINE#         282
  C:1F87H         LINE#         283
  C:1FA6H         LINE#         284
  C:1FC6H         LINE#         285
  C:1FE4H         LINE#         286
  C:1FF2H         LINE#         287
  C:1FF2H         LINE#         288
  -------         ENDPROC       _LCDDRAWCIRCLEA
  -------         PROC          _LCDCLEAR
  X:1DC0H         SYMBOL        color
  -------         DO            
  D:0004H         SYMBOL        i
  D:0002H         SYMBOL        j
  -------         ENDDO         
  C:4359H         LINE#         293
  C:4361H         LINE#         294
  C:4361H         LINE#         296
  C:4371H         LINE#         297
  C:4371H         LINE#         298
  C:4376H         LINE#         299
  C:4376H         LINE#         300
  C:4379H         LINE#         301
  C:437DH         LINE#         302
  C:4393H         LINE#         303
  C:4393H         LINE#         304
  C:439CH         LINE#         305
  C:43A3H         LINE#         306
  C:43AAH         LINE#         307
  -------         ENDPROC       _LCDCLEAR
  -------         PROC          _LCDSETPOS
  D:0002H         SYMBOL        x
  D:0004H         SYMBOL        y
  C:451EH         LINE#         311
  C:4522H         LINE#         312
  C:4522H         LINE#         313
  C:452AH         LINE#         314
  C:4530H         LINE#         315
  C:4536H         LINE#         316
  C:453CH         LINE#         318
  C:453FH         LINE#         319
  C:4540H         LINE#         320
  C:4543H         LINE#         321
  -------         ENDPROC       _LCDSETPOS
  -------         PROC          _LCDFILL
  X:1DC7H         SYMBOL        sx
  X:1DC9H         SYMBOL        sy
  D:0002H         SYMBOL        ex
  X:1DCDH         SYMBOL        ey
  X:1DCFH         SYMBOL        color
  -------         DO            
BL51 BANKED LINKER/LOCATER V6.22                                                      11/30/2016  13:53:19  PAGE 22


  X:1DD1H         SYMBOL        i
  D:0004H         SYMBOL        j
  X:1DD3H         SYMBOL        xlen
  -------         ENDDO         
  C:3F10H         LINE#         328
  C:3F1EH         LINE#         329
  C:3F1EH         LINE#         331
  C:3F25H         LINE#         333
  C:3F40H         LINE#         334
  C:3F65H         LINE#         335
  C:3F65H         LINE#         336
  C:3F70H         LINE#         337
  C:3F80H         LINE#         338
  C:3F80H         LINE#         339
  C:3F88H         LINE#         340
  C:3F90H         LINE#         341
  C:3F97H         LINE#         342
  C:3FA7H         LINE#         343
  -------         ENDPROC       _LCDFILL
  -------         PROC          _LCDSETBKCOLOR
  D:0006H         SYMBOL        color
  C:463CH         LINE#         347
  C:463CH         LINE#         348
  C:463CH         LINE#         349
  C:4644H         LINE#         350
  -------         ENDPROC       _LCDSETBKCOLOR
  -------         PROC          _LCDSETCOLOR
  D:0006H         SYMBOL        color
  C:4645H         LINE#         354
  C:4645H         LINE#         355
  C:4645H         LINE#         356
  C:464DH         LINE#         357
  -------         ENDPROC       _LCDSETCOLOR
  -------         PROC          _LCDDISPCHAR
  X:1DD2H         SYMBOL        x
  X:1DD4H         SYMBOL        y
  X:1DD6H         SYMBOL        ch
  X:1DD7H         SYMBOL        font
  X:1DD8H         SYMBOL        mode
  -------         DO            
  X:1DD9H         SYMBOL        temp
  X:1DDAH         SYMBOL        t1
  D:0001H         SYMBOL        t
  X:1DDBH         SYMBOL        y0
  X:1DDDH         SYMBOL        csize
  -------         ENDDO         
  C:353AH         LINE#         364
  C:354FH         LINE#         365
  C:354FH         LINE#         367
  C:3557H         LINE#         369
  C:357FH         LINE#         371
  C:3586H         LINE#         373
  C:3595H         LINE#         374
  C:3595H         LINE#         376
  C:35AFH         LINE#         377
  C:35D9H         LINE#         380
  C:35DEH         LINE#         381
BL51 BANKED LINKER/LOCATER V6.22                                                      11/30/2016  13:53:19  PAGE 23


  C:35DEH         LINE#         382
  C:35F8H         LINE#         383
  C:3612H         LINE#         384
  C:3619H         LINE#         385
  C:3627H         LINE#         387
  C:363DH         LINE#         388
  C:3659H         LINE#         389
  C:3659H         LINE#         390
  C:3661H         LINE#         391
  C:366FH         LINE#         393
  C:3685H         LINE#         395
  C:3685H         LINE#         396
  C:3694H         LINE#         397
  C:3698H         LINE#         398
  -------         ENDPROC       _LCDDISPCHAR
  -------         PROC          _LCDDISPSTRING
  X:1DC1H         SYMBOL        x
  X:1DC3H         SYMBOL        y
  X:1DC5H         SYMBOL        width
  X:1DC7H         SYMBOL        height
  X:1DC9H         SYMBOL        str
  X:1DCCH         SYMBOL        font
  X:1DCDH         SYMBOL        mode
  -------         DO            
  X:1DCEH         SYMBOL        x0
  X:1DD0H         SYMBOL        y0
  -------         ENDDO         
  C:3386H         LINE#         405
  C:339AH         LINE#         406
  C:339AH         LINE#         407
  C:33A9H         LINE#         408
  C:33B8H         LINE#         410
  C:33CBH         LINE#         411
  C:33CBH         LINE#         413
  C:33CEH         LINE#         414
  C:33CEH         LINE#         415
  C:33E0H         LINE#         416
  C:33EDH         LINE#         417
  C:33FCH         LINE#         418
  C:3402H         LINE#         419
  C:340CH         LINE#         420
  C:340EH         LINE#         421
  C:340EH         LINE#         423
  C:343FH         LINE#         424
  C:343FH         LINE#         425
  C:344EH         LINE#         426
  C:345DH         LINE#         427
  C:345DH         LINE#         428
  C:348EH         LINE#         429
  C:349FH         LINE#         430
  C:349FH         LINE#         431
  C:34B1H         LINE#         432
  C:34C0H         LINE#         433
  C:34CAH         LINE#         434
  C:34CAH         LINE#         435
  C:34FAH         LINE#         436
  C:3504H         LINE#         437
BL51 BANKED LINKER/LOCATER V6.22                                                      11/30/2016  13:53:19  PAGE 24


  C:3518H         LINE#         438
  C:351BH         LINE#         439
  C:352AH         LINE#         440
  C:3539H         LINE#         441
  -------         ENDPROC       _LCDDISPSTRING
  -------         PROC          _LCD_PRINTF
  X:1DFEH         SYMBOL        format
  -------         DO            
  X:1E01H         SYMBOL        ellipsis_40
  X:1E29H         SYMBOL        arg
  X:1E2CH         SYMBOL        tmp
  -------         ENDDO         
  C:3D9FH         LINE#         445
  C:3DAAH         LINE#         446
  C:3DAAH         LINE#         450
  C:3DC4H         LINE#         451
  C:3DCAH         LINE#         454
  C:3DD8H         LINE#         455
  C:3E10H         LINE#         463
  C:3E5BH         LINE#         466
  C:3E6BH         LINE#         467
  -------         ENDPROC       _LCD_PRINTF
  -------         ENDMOD        TFTLCD

  -------         MODULE        74HC165
  C:0000H         SYMBOL        _ICE_DUMMY_
  B:00B0H.5       PUBLIC        HC165_OUT
  D:00B0H         PUBLIC        P3
  C:456FH         PUBLIC        HC165_Read
  B:00B0H.4       PUBLIC        HC165_nPL
  B:00B0H.3       PUBLIC        HC165_CK
  -------         PROC          HC165_READ
  -------         DO            
  D:0006H         SYMBOL        i
  D:0007H         SYMBOL        Temp
  -------         ENDDO         
  C:456FH         LINE#         4
  C:456FH         LINE#         5
  C:456FH         LINE#         8
  C:4571H         LINE#         9
  C:4573H         LINE#         10
  C:4575H         LINE#         11
  C:4577H         LINE#         12
  C:457BH         LINE#         13
  C:457DH         LINE#         14
  C:457DH         LINE#         15
  C:457FH         LINE#         16
  C:4581H         LINE#         17
  C:4585H         LINE#         18
  C:4588H         LINE#         19
  C:4588H         LINE#         20
  C:458BH         LINE#         21
  C:458BH         LINE#         22
  C:4590H         LINE#         23
  C:4592H         LINE#         24
  C:4592H         LINE#         25
  -------         ENDPROC       HC165_READ
BL51 BANKED LINKER/LOCATER V6.22                                                      11/30/2016  13:53:19  PAGE 25


  -------         ENDMOD        74HC165

  -------         MODULE        ?C?SCDIV
  C:1FF3H         PUBLIC        ?C?SCDIV
  -------         ENDMOD        ?C?SCDIV

  -------         MODULE        ?C?CLDPTR
  C:2015H         PUBLIC        ?C?CLDPTR
  -------         ENDMOD        ?C?CLDPTR

  -------         MODULE        ?C?CSTPTR
  C:202EH         PUBLIC        ?C?CSTPTR
  -------         ENDMOD        ?C?CSTPTR

  -------         MODULE        ?C?IMUL
  C:2040H         PUBLIC        ?C?IMUL
  -------         ENDMOD        ?C?IMUL

  -------         MODULE        ?C?SIDIV
  C:2052H         PUBLIC        ?C?SIDIV
  -------         ENDMOD        ?C?SIDIV

  -------         MODULE        ?C?IILDX
  C:2088H         PUBLIC        ?C?IILDX
  -------         ENDMOD        ?C?IILDX

  -------         MODULE        ?C?ILDIX
  C:209EH         PUBLIC        ?C?ILDIX
  -------         ENDMOD        ?C?ILDIX

  -------         MODULE        ?C?ILDOPTR
  C:20B4H         PUBLIC        ?C?ILDOPTR
  -------         ENDMOD        ?C?ILDOPTR

  -------         MODULE        ?C?ISTOPTR
  C:20ECH         PUBLIC        ?C?ISTOPTR
  -------         ENDMOD        ?C?ISTOPTR

  -------         MODULE        ?C?LMUL
  C:2119H         PUBLIC        ?C?LMUL
  -------         ENDMOD        ?C?LMUL

  -------         MODULE        ?C?ULDIV
  C:21A4H         PUBLIC        ?C?ULDIV
  -------         ENDMOD        ?C?ULDIV

  -------         MODULE        ?C?ULCMP
  C:2236H         PUBLIC        ?C?ULCMP
  -------         ENDMOD        ?C?ULCMP

  -------         MODULE        ?C?LLDIXDATA
  C:2250H         PUBLIC        ?C?LLDIXDATA
  C:2247H         PUBLIC        ?C?LLDIXDATA1
  C:2249H         PUBLIC        ?C?LLDIXDATA8
  -------         ENDMOD        ?C?LLDIXDATA

  -------         MODULE        ?C?LSTXDATA
BL51 BANKED LINKER/LOCATER V6.22                                                      11/30/2016  13:53:19  PAGE 26


  C:227CH         PUBLIC        ?C?LSTXDATA
  -------         ENDMOD        ?C?LSTXDATA

  -------         MODULE        ?C?LSTKXDATA
  C:2288H         PUBLIC        ?C?LSTKXDATA
  -------         ENDMOD        ?C?LSTKXDATA

  -------         MODULE        ?C?ICALL
  C:22B9H         PUBLIC        ?C?ICALL
  C:22BDH         PUBLIC        ?C?ICALL2
  -------         ENDMOD        ?C?ICALL

  -------         MODULE        VSPRINTF
  X:1EC5H         PUBLIC        ?_VSPRINTF?BYTE
  C:43F5H         PUBLIC        _VSPRINTF
  -------         ENDMOD        VSPRINTF

  -------         MODULE        ?C?UIDIV
  C:22BFH         PUBLIC        ?C?UIDIV
  -------         ENDMOD        ?C?UIDIV

  -------         MODULE        PRINTF
  X:1E2FH         PUBLIC        ?_PRINTF517?BYTE
  X:1E2FH         PUBLIC        ?_PRINTF?BYTE
  X:1E2FH         PUBLIC        ?_SPRINTF517?BYTE
  X:1E2FH         PUBLIC        ?_SPRINTF?BYTE
  C:23F2H         PUBLIC        _PRINTF
  C:23F2H         PUBLIC        _PRINTF517
  C:23ECH         PUBLIC        _SPRINTF
  C:23ECH         PUBLIC        _SPRINTF517
  -------         ENDMOD        PRINTF

  -------         MODULE        ?C?CLDOPTR
  C:2314H         PUBLIC        ?C?CLDOPTR
  -------         ENDMOD        ?C?CLDOPTR

  -------         MODULE        ?C?PLDIXDATA
  C:2341H         PUBLIC        ?C?PLDIXDATA
  -------         ENDMOD        ?C?PLDIXDATA

  -------         MODULE        ?C?PSTXDATA
  C:2358H         PUBLIC        ?C?PSTXDATA
  -------         ENDMOD        ?C?PSTXDATA

  -------         MODULE        ?C?CCASE
  C:2361H         PUBLIC        ?C?CCASE
  -------         ENDMOD        ?C?CCASE

  -------         MODULE        PUTCHAR
  C:4548H         PUBLIC        _PUTCHAR
  -------         ENDMOD        PUTCHAR

Program Size: data=15.1 xdata=7886 code=17998
LINK/LOCATE RUN COMPLETE.  0 WARNING(S),  0 ERROR(S)
